:030000000219FDE5
:03000B000200AA46
:03002B0002015C73
:03005B000202F9A5
:030073000202E6A0
:1000800002030406080C10182030406080040608A3
:100090000C10182030406080A0C00003070F1F0D17
:1000A0000D04050D050305030302C2AFC0D0C0E077
:1000B000206214E5256009E473E525F4F58AD2622F
:1000C000D0E0D0D0D2AF3285268AC262E526F46075
:1000D0002F30682520720DD0E0D0D0D297D295D2A3
:1000E00093D2AF32D297D295D293206F0C2066096B
:1000F000740AD5E0FDE57B4290D0E0D0D0D2AF329B
:10010000758A00C28DD26201F901B9306805206696
:1001100002C29701B9306805206602C29501B93064
:100120006805206602C29301B9C29630680A20664B
:10013000077408D5E0FDC29701B9C29430680A205F
:1001400066077408D5E0FDC29501B9C29230680A0D
:100150002066077408D5E0FDC29301B9C2AFC2ADF5
:1001600053E6EFC0D0C0E0D2D3D2AFC2CEE52A6012
:1001700007207449152A21BD7800790020742EE5E6
:1001800080307E01F430E50278FF53DACF207E0321
:1001900043DA20307E0343DA10C2D8C271E58030E2
:1001A0007E01F430E50279FFC3E89970CB3061033A
:1001B000752A18207403752A18885CD27020740D73
:1001C000E52B6004152B21CD43DA01C2D820700243
:1001D000413CA85C206102C2702074367982B70469
:1001E00031C3E894F0400374F0F8E8C4540F28F8E1
:1001F0007984B703024112C313C313872120080275
:10020000C313200A06C3C898F8411228F850037493
:10021000FFF88822E52D54066022206B1FE536C3C7
:1002200033C333F8E564C313C313F9C39522400203
:100230008922E82522F52250037522FF7882B60430
:1002400059852224A824C3E52495614002A861C3EE
:10025000E895634002A8638825E5667002418DC376
:10026000E8AA669A5003E8FAE4F9EAC333FBE568C2
:10027000F45B29400D2567F8E56760021567400BC0
:10028000418D0AC3E5679A5002056778FF8826C248
:100290006FC3E52694F84002D26FC3E52594404031
:1002A00002D26420CF0AD0E0D0D043E610D2AD32E3
:1002B000C2CF053A7801E52A6005307402152AC3D9
:1002C000E55C94014005755F0041DC75600075696F
:1002D00000E55F2401F55F5003755FFFD0E0D0D0EB
:1002E00043E610D2AD32C2AF53E67F7592FA7593F2
:1002F000FFC260759104D2AF32C2AF53E6EFC2AD18
:10030000C0D0C0E0C0F0D2D3D2AFA8FBA9FCC2D805
:10031000307102616053DACF207E0343DA10307E01
:100320000343DA20D271E580307E01F420E50261DA
:100330003788278928A18D53DACF207E0343DA201E
:10034000307E0343DA10C2D8C271307402A17978CA
:1003500000E580307E01F430E502A179885CA1617E
:1003600053DACF207E0343DA20307E0343DA10C213
:1003700071206102813953DACF207E0343DA1030D5
:100380007E0343DA20C2D8D27188578958C3E895D2
:1003900055F8E99556F97B007E087A00C3E8948CFD
:1003A000E994005005755B00812B882178A2E6A8AE
:1003B000216055C3E894C8E994005008E4D2E4FBF6
:1003C0007A0A8106C3E89468E994015008E4D2E30C
:1003D000FB7A0F8106C3E894D0E994025008E4D276
:1003E000E2FB7A1E8106C3E894A0E994055008E474
:1003F000D2E1FB7A3C8106C3E89498E9940850085E
:10040000E4D2E0FB7A787E00C3E89559FCE9955A7E
:10041000FD30E70AECF42401FCEDF43400FD755BDB
:1004200000C3EC9AED9E5003755B018859895A858B
:1004300057558558567802A161C3E89527F8E99584
:1004400028F9307C02A145307B02A145307A02A117
:100450003E207502815CE9FDE8FC817BE9C313F96C
:10046000E813F8307902A13EE9C313F9E813F83034
:0F0470007802A13EE9C313FDE813FC20612CC301
:10047F00EC941CED940240028192ED701EC3EC943B
:10048F00C850180529E52970021529C3E529940AD2
:10049F005002A179755C00D270A179E5296002152F
:1004AF00297888E6F97400207F087896B9030278D6
:1004BF009EE624FAFEE43400FFC3EC9EFCED9FFDA4
:1004CF009208B90310A2085007207609D27681E46A
:1004DF00307602C276A2085016B9030DECF424014F
:1004EF00FCEDF43400FD0204FE78007900A145B95B
:1004FF000315EC33FCED33FDC3EC940AFCED9400D3
:10050F00FD50047C007D00C3EC94FFED9400400689
:10051F0078FF7900A145EC8572F0A4C5F0A2F733FE
:10052F00F87900400302056178FF7900020561E95F
:10053F00C313F9E813F8307C0EE9600278FFC3E8C3
:10054F001338F8E43400F9C3E894FFE9940040024B
:10055F0078FF885CD270206102A179741FF4552F47
:10056F004BF52FC274EB7002D274752A18307403D6
:10057F00752A0A306102A18D20740353DAFE2074AC
:10058F0003752B06D0F0D0E0D0D0D2AD43E61032B9
:10059F0079010205BD79030205BD790A0205BD790E
:1005AF001E0205BD79640205BD79C80205BD781725
:1005BF00E4D5E0FDD8FAD9F6227A147B780205E467
:1005CF007A107B8C0205E47A0D7BB40205E47A0B7A
:1005DF007BC80205E47902E4C294D5E0FDC295D54B
:1005EF00E0FDD295D5E0FDD294D5E0FDE920E00203
:1005FF00C29730E002C293E573D5E0FDE920E00237
:10060F00D29730E002D2937496D5E0FDD9C9EAF8BB
:10061F00D5E0FDD8FBDBBEC29422C37C007D007504
:10062F00F00005F0EA33FAEB33FB50F6EB13FBEA7D
:10063F0013FAC3E9FFE8FEE89AF8E99BF95004EFD3
:10064F00F9EEF8B3EC33FCED33FDD5F0DFEDF9EC5B
:10065F00F822E889F08A20D2D4F8A9F07B0030F78D
:10066F000B7BFFF42401F8E9F43400F9E88520F05E
:10067F00A4ADF0F8E98520F0A4AFF0FEED2EF974EB
:10068F00003FFA7C04C3EA13FAE913F9E813F8DC24
:10069F00F48BF030F70AE8F42401F8E9F43400F9A8
:1006AF00E889F0C2D4F8A9F0227882B604030207D1
:1006BF0013C3E55C940140030206DD852224E4F5B3
:1006CF0044F545F546F547F548C26E0207137882A3
:1006DF00E6FCD26EE522F523783879C7AA40AB4104
:1006EF00C3EB13FBEA13FAEC146013C3EB13FBEA2F
:1006FF0013FAEC14146007C3EB13FBEA13FAD129B6
:10070F008844894522C3E5449523F8E5459400F9CB
:10071F00500CC3E89480E994FF4016020744C3E8E5
:10072F00947FE994005003020744787F7900020711
:10073F0044788079FF8849894A22E5492546F8E5BA
:10074F004A3547F9854A20E4300701F43548FA3035
:10075F00E709C3EA94F04015020782C3EA940F50E9
:10076F000302078278FF79FF7A0F020782780079F8
:10077F00007AF0C3E5249561500AC37401952450A3
:10078F000B0207A0E54A20E70E0207A0E54A30E773
:10079F0006884689478A482278A5E6FAC3E5493391
:1007AF00F8E54A33F9D161E930E70BC3E89480E902
:1007BF0094FF4013E1DAC3E8947FE994005002E11B
:1007CF00DA787F7900E1DA788079FFE820E715C3DE
:1007DF00E52398F84009C3E8940140030208017823
:1007EF0001020801E8F424012523F840030208015F
:1007FF0078FF884B2278A6E6FAA847A94812066127
:10080F00E930E70CC3E89401E994FF40160208367B
:10081F00C3E894FFE99400500302083678FF79008B
:10082F00020836780179FFE920E715C3E54B98F800
:10083F004009C3E89401400302085D780102085D96
:10084F00E8F42401254BF8400302085D78FF882463
:10085F002278FFC26420693D206A12D264C3E54149
:0F086F00940A4009C3E52594405002C26479A160
:10087E00E76023E541601F74FF8541F0848539F000
:10088E00306A0375F005A4F8C5F0600278FFC3E87E
:10089E0095645002A864886322C3E5409440E54104
:1008AE009401E56350031401B8046002F56322025B
:1008BE0008C02275E890227883E6FFE5E820ECF781
:1008CE00A8BDA9BE0570C3E57094084052757000AE
:1008DE00E9FA79A0E76044EA7007E571601B020847
:1008EE00FBC3E895716010E5715006600C140209A7
:1008FE00070460F9020907E571F571C3946D401B99
:10090E007561C0C394044013756180C39404400B99
:10091E00756140C39404400375610075BB0822E500
:10092E00612410500274FFF5617982B704022154DC
:10093E00C3A861E524985002A824C3E89563400239
:10094E00A86388258826E570B4070375BB1022744A
:10095E003279A787F0A4C5F0A2F733F8C3E8956102
:10096E004002A861882288248825882688642275FA
:10097E0040007541F022C2AF75C820A8CCA9CDAAFF
:10098E003A30CF010A75C824D2AFAB3BAC3C883BA2
:10099E00893CC3E89BF8E99C206908F9306702415D
:1009AE009021EDAD3D8A3DF9EA9DFA600478FF791C
:1009BE00FFAE3EAF3F8B3E8C3FA83BA93CC3E89EAB
:1009CE00F8E99FF9C3E54113FBE54013FAE82AF570
:1009DE0040E93BF54150067540FF7541FF4137AA8E
:1009EE0040AB41AC40AD417E047F02C3EB9404406A
:1009FE00021E1FC3EB940840021E1FC3ED13FDEC35
:100A0E0013FCDEF7C3EA9CFAEB9DFBEF6009C3E92A
:100A1E0013F9E813F8DFF7EA28FAEB39FB8A408B73
:100A2E004150067BFF8B408B41C3EB94025002D2A8
:100A3E00673069047F0341627892E6FFC3E537941D
:100A4E008240110FC3E53794A040010FC3EF940607
:100A5E0040027F057E02E541C4540FF9E541C454BE
:100A6E00F0F8E540C4540F28F8C3E89EFAE9940064
:100A7E00FB4009C3EA9402EB940050047A02E4FBB3
:100A8E0041DCAA40AB41EBC4FEEAC4540F4EFCC39A
:100A9E00EA9CFAEB9400FBC3E813C313F8EA28FAB6
:100AAE00EB3400FB8A408B41C3EB94024002C267D9
:100ABE007802EBC4FE7B00EAC4540F4EFAC3EA98E8
:100ACE00FA4005C3940250027A027892E6FF306033
:100ADE000241DC855192855293D26043E680C3E495
:100AEE009AF8E49BF93067026168E8FAE9FBD3E90A
:100AFE0013FDE813FC88518952C3EF94036038EF5D
:100B0E0020E00DE82CF8E93DF9ECFAEDFB020B3193
:100B1E00E828F8E939F9C3E82402F8E93400F97A4B
:100B2E00FE7BFFC3EF9403400E8A538B54884D898E
:100B3E004E8C4F8D50619C885389548A4D8B4E8CB0
:100B4E004F8D503069127553F07554FF754FF07517
:100B5E0050FF7551F07552FF619CE8FAD3E813FC13
:100B6E008851C3EF94036020EF20E007E82CF8ECE7
:100B7E00FA6188E8282402F87AFEC3EF940340084D
:100B8E008A53884D8C4F619C88538A4D8C4FE568F3
:100B9E00C3335002646BF56830600261A67534028F
:100BAE00D26043E680E52D54066034A840A941C3C7
:100BBE00E913F9E813F8C3E913F9E813F8306904F7
:100BCE00E92440F9C2AF53E67F759100C3E498F56E
:100BDE0094E499F595759104D26043E680D2AF22E4
:100BEE00D265754300752000306C03752040020CF1
:100BFE000DD265754300752040306C03752000786A
:100C0E00017901206720E52D54066002C265791432
:100C1E00E541C313700104F8C394144002781430F4
:100C2E006904781B791B206010E543600C30690362
:100C3E00D53404D26D81AF71AE0543E59B5440B5FA
:100C4E002002819930690908C3E89940011881345E
:100C5E0020650A08C3E8994002810D8134C265C23D
:0D0C6E00AF53E67F7591003067127594005A
:100C7B007595FE759104D26043E680D2AF810DAEBF
:100C8B0040AF41C3E49EF594E49FF595817EC3E5A7
:100C9B003394015002810D306502810DD80281AD74
:100CAB008134C26DC2AF53E67F7591008553948535
:100CBB005495759104854D92854E93D26043E68091
:100CCB00D2AFE52D54066008206A020533020CEB07
:100CDB00306D0D206C0A2065071581158102157387
:100CEB002278003064053065027801E53775F0072E
:100CFB00A4F9E5F028F5F0E9A2F013A2F113A2F2A2
:100D0B0013F537C394785003753778C3E5379538A7
:100D1B004008D266D297D295D293306002A1258536
:100D2B004F92855093D26043E68022207D16C2AF4E
:100D3B00754202C294D296306202C293D2AF759FB3
:100D4B0010020F25C2AF754202C294D292306202DA
:100D5B00C297D2AF759F10020F25307243207D20B2
:100D6B00C2AF75420390013A757B10D293C2923099
:100D7B006204C295A183D294D2AF759F13020F2543
:100D8B00C2AF75420390013A757B10D297C2963071
:100D9B006204C295A1A3D294D2AF759F11020F2505
:100DAB00207D17C2AF754203900115D293306202BA
:100DBB00C295D2AF759F13020F25C2AF7542039038
:100DCB000115D297306202C295D2AF759F11020FF7
:100DDB0025207D16C2AF754204C296D292306202B4
:100DEB00C295D2AF759F11020F25C2AF754204C2D7
:100DFB0092D296306202C295D2AF759F13020F2525
:100E0B00307243207D20C2AF754205900129757B5E
:100E1B0040D295C294306204C297C129D296D2AF08
:100E2B00759F10020F25C2AF75420590014B757B64
:100E3B0004D295C294306204C293C149D292D2AF0C
:100E4B00759F10020F25207D17C2AF7542059001CB
:100E5B000BD295306202C297D2AF759F10020F254D
:100E6B00C2AF75420590011FD2953062EBC293D28F
:100E7B00AF759F10020F25207D16C2AF754206C2BB
:100E8B0092D294306202C297D2AF759F13020F2594
:100E9B00C2AF754206C296D294306202C293D2AFF1
:100EAB00759F11020F25307243207D20C2AF754212
:100EBB000190014B757B04D297C296306204C293AA
:100ECB00C1CFD292D2AF759F11020F25C2AF75421F
:100EDB0001900129757B40D293C292306204C29774
:100EEB00C1EFD296D2AF759F13020F25207D17C28B
:100EFB00AF75420190011FD297306202C293D2AFFD
:100F0B00759F11020F25C2AF75420190010BD29351
:100F1B00306202C297D2AF759F13C266229001094D
:100F2B00757B00D297D295D293C296C294C292C2CD
:100F3B006222788076090876090876040876FF081D
:100F4B0076030876FF08760A08760308760108769A
:100F5B0001788C76010876FF0876FF0876FF087615
:100F6B00FF0876FF0876030876FF0876FF0876FF02
:100F7B000876250876D00876280876500876040877
:100F8B0076FF08760208760008767A0876FF0876F0
:100F9B000108760108760008760308760022788728
:100FAB00E6FFC272BF0302D2727888E6C394036075
:100FBB0008C27DE630E102D27DC27E7889E630E15F
:100FCB0002D27EC3EF94026008758E01D273020FBA
:100FDB00E1758E00C273227880E6149000809378BE
:100FEB00A5F67881E6149000809378A6F67886E6CD
:100FFB001490008D9378A7F67886E6F539C39402A2
:10100B005003753902789CE67538FFB402037538C6
:10101B00A0B4030375388278A3E61490009A93F575
:10102B0066120F2822227896E6FA7897E6FB7888E4
:10103B00E6B40305C3EB940EFB307F047A007BFF11
:10104B00C3EB9AFCC3948250027C827572000572CA
:10105B00EC8572F0A4C3E5F0947D40F222D27F11AF
:0F106B00311205AE7A007B007C101205A4E55C03
:10107A002AFA74003BFBDCF37C04C3EB13FBEA1390
:10108A00FADCF7FEC27F113122E5EF20E603752074
:10109A00000520903FFFE520146006901DFF1460B4
:1010AA00009304600375EF1253D9BF7581C043FFE3
:1010BA008012059F75EF0243B203E5B3240220E7CD
:1010CA000DF521E5E320E0068521B343E301120F84
:1010DA00287580FF75A40075F1B275D4DF7590A9E3
:1010EA0075A5FC75F2FC75D50175A60175E241126C
:1010FA000F28E4F8F6D8FD756801120F3D1215C4E1
:10110A0078988673753001C2AF1205B81205C812F5
:10111A0005AE1205CF1205AE1205D61205AEC2AF44
:10112A0078FA79FA308507D9FBD8F7021C00120F32
:10113A00A9120FE21130113178988673120F2875AF
:10114A00881075890275C82475910475D84075A8E8
:10115A002275B80275E690759B80759D0075D10E53
:10116A0075BC5875BB0875BA1175E88012059FD20F
:10117A00AF1208BD75360053DACF207E0343DA205A
:10118A00307E0343DA1043DA01C2D8C2711205B8BD
:10119A00D2617B037A0CE55B70077A0CDB030211E0
:1011AA00281205AE207003021128C270E55CC394B0
:1011BA000240E1E52F541F855E5DF55EB55DD5DA27
:1011CA00D5C26153DACF207E0343DA20307E03434F
:1011DA00DA10C2D8C27178A2E67008D274E52F5428
:1011EA00E0F52FC2757529001205B3307409C3E5FD
:1011FA0029940A4002D2751205A478023074027842
:10120A0000C3E55C9840F0C2AF1205C81205C812C7
:10121A0005C8D2AF1205B8754C007888E6B4030247
:10122A0061001205A4788CE6C394015003021300EE
:10123A00E530C394015003021300207435C3E55C02
:10124A0094FF5003021300C2AF1205DDD2AF12059C
:10125A00B3C3E55C940150EFC2AF1205C81205A9E9
:10126A001205C8D2AF1205B3C3E55C94FF40E90288
:10127A00176C7F02D27F11311205B3C2AFC27F1140
:10128A0031AE5CC3E55C947FD2AF407412059FC255
:10129A00AF1205DDD2AFDFDC1168C3EE7897F61224
:1012AA0005B81216061216EF7F0AD27F11311205FF
:1012BA00B3C2AFC27F1131AE5CC3E55C947FD2AFDB
:1012CA0050E612059FC2AF1205C81205A91205C839
:1012DA00D2AFDFD61168EE24037896F61205B8125B
:1012EA00160612171E1205B31131C3E55C94FF509E
:1012FA0002414402176CC3E55C954C4003855C4C83
:10130A001205B378017988E7B403027805C3E55C6E
:10131A009840024124C2AF1205DD1205DD1205DD37
:10132A00D2AF1205B8753000E4F531F5320531E572
:10133A0031F4703F0532789AE678191460127832DF
:10134A0014600D787D14600878FA14600375320011
:10135A00C3E53298401D120F2812059F15327531C8
:10136A000078998673C2AF1205DDD2AF789886737A
:10137A001205B31205A9E52A7005307402212878EE
:10138A00012074027806C3E55C9840A17888E6C318
:10139A00940360031205B3E52A7003021128C2AF51
:1013AA00120F28E4F522F523F524F525F526F5672D
:1013BA00D2AF7885E6C333F565E4F544F545F546DD
:1013CA00F547F548F570F52CF52DF5377570087564
:1013DA00BB1012059F1208C1E5E820ECFBA8BDA9C5
:1013EA00BEE97001F888711208C575700875BB10DE
:1013FA00120FA9C2AF7561FF12095D8522618522AC
:10140A0062852263D2AF75220175240175250175A3
:10141A002601856069756A017888E6B40307C27D8A
:10142A00307602D27DD268D269753300120E8212EA
:10143A000EB112097D12098412097D12098412095A
:10144A007D120BFF1206B8120CEC120D361209842B
:10145A00120BEE306E031207142067031208603075
:0E146A0067031208A7120CEC120D651209841C
:10147800120BFF306E03120749120CEC120DDC122E
:101488000984120BEE306E031207A7120CEC120E31
:101498000B120984120BFF306E03120804120CECB5
:1014A800120E821209841208C1120BEE120CEC12F1
:1014B8000EB11208C51209843069328564618564E9
:1014C80062856069756A0179187A0CC3E5339940B9
:1014D8000FC269D26A8A358564618564630214F52E
:1014E800C3E55C9401400302144B02157B306A1D6E
:1014F800206C1AE535147006C26AD26B814BF5353B
:10150800C3E55C9401400302144B02157B75360059
:1015180078FA79A4E760027803C3E55F98505430FD
:101528007404E52A604D7888E6B40317207D052009
:101538007607A14B307602A14B206C07D26C8564EC
:1015480061818A78F0306C058564617820C3E54153
:10155800985002814B306C1BC26CC27D307602D22F
:101568007DD26A753512856461814B0536E55C600C
:1015780002A17E753600C2AF120F287887E6FE7684
:1015880002120FA97887EEF6E4F522F523F524F583
:1015980025F526F565752C00752D00D2AF1205B31B
:1015A800120F2878A4E66006C297C295C2933074D9
:1015B80009C3E5369404400221286132901A0D7857
:1015C80020121648E520B4550CA3121648E520B49D
:1015D800AA030215E6120F3D121606021605901A06
:1015E8000378807B0A121648A308DBF9901A0F7853
:1015F8008C7B19121648A308DBF9901A2822C2AF6F
:10160800121687121661901A00740E12164DA374E2
:101618000612164DA3741512164D901A0378807B86
:101628000A12164CA308DBF9901A0F788C7B191252
:10163800164CA308DBF912169A121678901A28226B
:10164800E493F622E6438F01538FFD75EF0275B7D9
:10165800A575B7F1F0538FFE22438F02438F0175B2
:10166800EF0275B7A575B7F1901A0DF0538FFC22EC
:10167800901A0D7455D14D901A0E74AAD14D227A34
:101688003079D07820901A40D148E520F709A3DABC
:10169800F7227A3079D0901A40E7D14D09A3DAF9C8
:1016A80022AB74A875BB01027980BB02027981BBA9
:1016B80003027982BB04027984BB05027986BB06E2
:1016C800027992BB07027987BB080279A3BB09029A
:1016D800799CBB0A027988BB0B027989E8F7227CDE
:1016E800051205B8DCFB22C2AF1205C81205CF12DD
:1016F80005D61205DD1205A91205C81205CF120577
:10170800D61205DD1205A91205C81205CF1205D695
:101718001205DDD2AF22C2AF1205DD1205D61205C1
:10172800CF1205C81205A91205DD1205D61205CF7C
:101738001205C81205A91205DD1205D61205CF1229
:1017480005C8D2AF22AE74AF75C2AF1205C8120574
:10175800C81205C81205A9DEF21205DD1205A9DFB7
:10176800F8D2AF22D1EFD1E7D1E7757401757501D1
:10177800757600F14D7C05AD5C1205B8C3ED955C3E
:1017880070F5C3E55C9401400AC3E55C94FF403200
:101798000217A8D1A9D106D1EFC2AF75EF12D1E7D0
:1017A800DCD50576C3E5769403500280C6D1E705FB
:1017B80075E5741490009F93F808C3E57598500276
:1017C80080AED1E7D1E70574C3E574940C5002806C
:0D17D8009C120F3DD106C2AF75EF12D1E794
:0319FD0002109342
:101A00000E0615090904FF03FF0A03010155AA0187
:101A1000FFFFFFFFFF03FFFFFF25D0285004FF0259
:091A2000007AFF0101000300FF40
:101A400023536B7977616C6B6572323041232020B0
:101A500023424C48454C4923463333302320202031
:101A60002020202020202020202020202020202076
:101C0000C2AFC2D353D9BF7581C043B20343FF8073
:101C1000752438752503B1C975EF0275E24043F1AB
:101C20002053A4DF75D4FFD2857DFA780379E67C52
:101C300010752200752300901DD67B0675249875BB
:101C400025013085028142208508D8FBD9F9DCF7CF
:101C500081B4308508D8FBD9F9DCF781B4B189E4C7
:101C600093A3C39A6004DDC381B4DBDBB17B600264
:101C7000812B7B08E493FAA3B15CDBF87A30B15C8A
:101C8000752200752300B17BEAFCEBFDC3ED94FEE9
:101C9000400EB17B8A278B28ED30E0048A828B834B
:101CA000B17B7AC270D8C3ED94FE601350CEBD00F4
:101CB00025EC60097520007521FF0200008100A855
:101CC00027A9280809D804D90281D3B17FEA89AAB3
:101CD000F281C50D81A0C3ED94035049EDA2E092BD
:101CE000007AC5C3E5829400E583941C50902000DF
:101CF00010438F02438F0175B7A575B7F1F030001F
:101D00001FA827A9280809438F01538FFDD804D99C
:101D100002A12089AAE275B7A575B7F1F0A3A10DBC
:101D2000538FFC817C7AC1BD030CE493A3FAB140CC
:101D3000DCF8B138817C817EAA22AB23B15CEBFA5E
:101D4000EA6222752608C3E52313F523E52213F57D
:101D50002250066323A0632201D526EAB1C9B1C986
:101D600075260AEAF4200102D285300102C285B14B
:101D7000C9C3134002C201D526EB22B17FEAFB2082
:101D80008502A17F308502A184752608AE24AF2587
:101D9000C3EF13FFEE13FEB1CDB1C9C3EA13308513
:101DA000024480FA30E703632201C3E52313F523DD
:101DB000E52213F52250066323A0632201D526D91C
:101DC000E52265236523F52222AE24AF250E0FDE22
:101DD000FEDFFCD20122424C48656C693437316326
:041DE000F3300601D5
:00000001FF
